 battdrvr

 Timestamp is 4da293c5 (Mon Apr 11 17:38:13 2011)

 Preferred load address is 10000000

 Start         Length     Name                   Class
 0001:00000000 00000004H .CRT$XCA                CODE
 0001:00000004 00000004H .CRT$XCZ                CODE
 0001:00000008 00000004H .CRT$XIA                CODE
 0001:0000000c 00000004H .CRT$XIZ                CODE
 0001:00000010 00000004H .CRT$XPA                CODE
 0001:00000014 00000004H .CRT$XPZ                CODE
 0001:00000018 00000004H .CRT$XTA                CODE
 0001:0000001c 00000004H .CRT$XTZ                CODE
 0001:00000020 000000a4H .rdata                  CODE
 0001:000000c4 00000025H .rdata$debug            CODE
 0001:000000ec 0000158cH .text                   CODE
 0001:00001678 00000114H .xdata                  CODE
 0001:0000178c 00000014H .idata$2                CODE
 0001:000017a0 00000014H .idata$3                CODE
 0001:000017b4 0000008cH .idata$4                CODE
 0001:00001840 0000000cH .idata$6                CODE
 0001:00001850 000000dcH .edata                  CODE
 0002:00000000 0000008cH .idata$5                DATA
 0002:0000008c 00000008H .data                   DATA
 0002:000000a0 000000f4H .bss                    DATA
 0003:00000000 00000188H .pdata                  DATA

  Address         Publics by Value              Rva+Base       Lib:Object

 0000:00000000       ___safe_se_handler_count   00000000     <absolute>
 0000:00000000       ___safe_se_handler_table   00000000     <absolute>
 0001:00000000       __xc_a                     10001000     corelib0:crt0init.obj
 0001:00000004       __xc_z                     10001004     corelib0:crt0init.obj
 0001:00000008       __xi_a                     10001008     corelib0:crt0init.obj
 0001:0000000c       __xi_z                     1000100c     corelib0:crt0init.obj
 0001:00000010       __xp_a                     10001010     corelib0:crt0init.obj
 0001:00000014       __xp_z                     10001014     corelib0:crt0init.obj
 0001:00000018       __xt_a                     10001018     corelib0:crt0init.obj
 0001:0000001c       __xt_z                     1000101c     corelib0:crt0init.obj
 0001:0000003c       ??_C@_1BM@KBMAGFOO@?$AAP?$AAd?$AAd?$AAB?$AAu?$AAf?$AAf?$AAe?$AAr?$AAS?$AAi?$AAz?$AAe?$AA?$AA@ 1000103c     battdrvr_mdd:battdrvr.obj
 0001:00000058       ??_C@_1BK@GMCBNGHD@?$AAP?$AAo?$AAl?$AAl?$AAI?$AAn?$AAt?$AAe?$AAr?$AAv?$AAa?$AAl?$AA?$AA@ 10001058     battdrvr_mdd:battdrvr.obj
 0001:00000074       ??_C@_1CA@NFABIDNC@?$AAP?$AAo?$AAl?$AAl?$AAP?$AAr?$AAi?$AAo?$AAr?$AAi?$AAt?$AAy?$AA2?$AA5?$AA6?$AA?$AA@ 10001074     battdrvr_mdd:battdrvr.obj
 0001:00000094       ??_C@_1DA@IBFGCKKH@?$AAS?$AAY?$AAS?$AAT?$AAE?$AAM?$AA?1?$AAB?$AAa?$AAt?$AAt?$AAe?$AAr?$AAy?$AAA?$AAP?$AAI?$AAs?$AAR?$AAe?$AAa?$AAd?$AAy?$AA?$AA@ 10001094     battdrvr_mdd:battdrvr.obj
 0001:000000ec       BatteryPDDInitialize       100010ec f   battdrvr.obj
 0001:000000f4       BatteryPDDDeinitialize     100010f4 f   battdrvr.obj
 0001:000000f8       BatteryPDDResume           100010f8 f   battdrvr.obj
 0001:000000fc       BatteryPDDPowerHandler     100010fc f   battdrvr.obj
 0001:00000100       BatteryPDDGetStatus        10001100 f   battdrvr.obj
 0001:00000120       BatteryPDDGetLevels        10001120 f   battdrvr.obj
 0001:00000128       BatteryPDDSupportsChangeNotification 10001128 f   battdrvr.obj
 0001:00000130       BatteryThreadProc          10001130 f   battdrvr_mdd:battdrvr.obj
 0001:00000214       Init                       10001214 f   battdrvr_mdd:battdrvr.obj
 0001:0000056c       PostInit                   1000156c f   battdrvr_mdd:battdrvr.obj
 0001:000005c0       Deinit                     100015c0 f   battdrvr_mdd:battdrvr.obj
 0001:0000069c       IOControl                  1000169c f   battdrvr_mdd:battdrvr.obj
 0001:00000c5c       PowerDown                  10001c5c f   battdrvr_mdd:battdrvr.obj
 0001:00000c64       PowerUp                    10001c64 f   battdrvr_mdd:battdrvr.obj
 0001:00000c88       Open                       10001c88 f   battdrvr_mdd:battdrvr.obj
 0001:00000c8c       Close                      10001c8c f   battdrvr_mdd:battdrvr.obj
 0001:00000c94       Read                       10001c94 f   battdrvr_mdd:battdrvr.obj
 0001:00000ca8       Write                      10001ca8 f   battdrvr_mdd:battdrvr.obj
 0001:00000cbc       Seek                       10001cbc f   battdrvr_mdd:battdrvr.obj
 0001:00000cc4       DllMain                    10001cc4 f   battdrvr_mdd:battdrvr.obj
 0001:00000cd8       BatteryAPIStopwatch        10001cd8 f   battdrvr_mdd:battapi.obj
 0001:00000dac       BatteryAPIGetSystemPowerStatusEx2 10001dac f   battdrvr_mdd:battapi.obj
 0001:00000fec       BatteryAPIGetSystemPowerStatusEx 10001fec f   battdrvr_mdd:battapi.obj
 0001:00001020       BatteryAPIGetLifeTimeInfo  10002020 f   battdrvr_mdd:battapi.obj
 0001:000010e8       BatteryAPINotifyOfTimeChange 100020e8 f   battdrvr_mdd:battapi.obj
 0001:00001180       EventModify                10002180 f   coredll:COREDLL.dll
 0001:00001190       WaitForSingleObject        10002190 f   coredll:COREDLL.dll
 0001:000011a0       PowerPolicyNotify          100021a0 f   coredll:COREDLL.dll
 0001:000011b0       CeSetThreadPriority        100021b0 f   coredll:COREDLL.dll
 0001:000011c0       DeleteCriticalSection      100021c0 f   coredll:COREDLL.dll
 0001:000011d0       CloseHandle                100021d0 f   coredll:COREDLL.dll
 0001:000011e0       LocalFree                  100021e0 f   coredll:COREDLL.dll
 0001:000011f0       CreateThread               100021f0 f   coredll:COREDLL.dll
 0001:00001200       LocalAlloc                 10002200 f   coredll:COREDLL.dll
 0001:00001210       RegCloseKey                10002210 f   coredll:COREDLL.dll
 0001:00001220       RegQueryValueExW           10002220 f   coredll:COREDLL.dll
 0001:00001230       OpenDeviceKey              10002230 f   coredll:COREDLL.dll
 0001:00001240       CreateEventW               10002240 f   coredll:COREDLL.dll
 0001:00001250       InitializeCriticalSection  10002250 f   coredll:COREDLL.dll
 0001:00001260       OpenEventW                 10002260 f   coredll:COREDLL.dll
 0001:00001270       ResumeThread               10002270 f   coredll:COREDLL.dll
 0001:00001280       GetLastError               10002280 f   coredll:COREDLL.dll
 0001:00001290       LeaveCriticalSection       10002290 f   coredll:COREDLL.dll
 0001:000012a0       EnterCriticalSection       100022a0 f   coredll:COREDLL.dll
 0001:000012b0       SetLastError               100022b0 f   coredll:COREDLL.dll
 0001:000012c0       CeSetPowerOnEvent          100022c0 f   coredll:COREDLL.dll
 0001:000012d0       DisableThreadLibraryCalls  100022d0 f   coredll:COREDLL.dll
 0001:000012e0       GetTickCount               100022e0 f   coredll:COREDLL.dll
 0001:000012f0       SystemTimeToFileTime       100022f0 f   coredll:COREDLL.dll
 0001:00001300       GetLocalTime               10002300 f   coredll:COREDLL.dll
 0001:00001310       FileTimeToSystemTime       10002310 f   coredll:COREDLL.dll
 0001:00001418       _DllMainCRTStartup         10002418 f   corelib0:pegdmain.obj
 0001:00001504       _cexit                     10002504 f   corelib0:cexit.obj
 0001:00001514       _initterm                  10002514 f   corelib0:crt0dat.obj
 0001:00001540       _cinit                     10002540 f   corelib0:crt0dat.obj
 0001:000015a0       __security_init_cookie     100025a0 f   corelib0:seccinit.obj
 0001:000015ec       __crt_ExitProcess          100025ec f   corelib0:exitproc_proxy.obj
 0001:000015f8       memcpy                     100025f8 f   corelib1:COREDLL.dll
 0001:00001608       memcmp                     10002608 f   corelib1:COREDLL.dll
 0001:00001618       memset                     10002618 f   corelib1:COREDLL.dll
 0001:00001628       __C_specific_handler       10002628 f   corelib1:COREDLL.dll
 0001:00001638       _XcptFilter                10002638 f   corelib1:COREDLL.dll
 0001:00001648       free                       10002648 f   corelib1:COREDLL.dll
 0001:00001658       __security_gen_cookie2     10002658 f   corelib1:COREDLL.dll
 0001:00001668       TerminateProcess           10002668 f   coredll:COREDLL.dll
 0001:0000178c       __IMPORT_DESCRIPTOR_COREDLL 1000278c     coredll:COREDLL.dll
 0001:000017a0       __NULL_IMPORT_DESCRIPTOR   100027a0     coredll:COREDLL.dll
 0002:00000000       __imp_EventModify          10003000     coredll:COREDLL.dll
 0002:00000004       __imp_WaitForSingleObject  10003004     coredll:COREDLL.dll
 0002:00000008       __imp_PowerPolicyNotify    10003008     coredll:COREDLL.dll
 0002:0000000c       __imp_CeSetThreadPriority  1000300c     coredll:COREDLL.dll
 0002:00000010       __imp_DeleteCriticalSection 10003010     coredll:COREDLL.dll
 0002:00000014       __imp_CloseHandle          10003014     coredll:COREDLL.dll
 0002:00000018       __imp_LocalFree            10003018     coredll:COREDLL.dll
 0002:0000001c       __imp_CreateThread         1000301c     coredll:COREDLL.dll
 0002:00000020       __imp_LocalAlloc           10003020     coredll:COREDLL.dll
 0002:00000024       __imp_RegCloseKey          10003024     coredll:COREDLL.dll
 0002:00000028       __imp_RegQueryValueExW     10003028     coredll:COREDLL.dll
 0002:0000002c       __imp_OpenDeviceKey        1000302c     coredll:COREDLL.dll
 0002:00000030       __imp_CreateEventW         10003030     coredll:COREDLL.dll
 0002:00000034       __imp_InitializeCriticalSection 10003034     coredll:COREDLL.dll
 0002:00000038       __imp_OpenEventW           10003038     coredll:COREDLL.dll
 0002:0000003c       __imp_ResumeThread         1000303c     coredll:COREDLL.dll
 0002:00000040       __imp_GetLastError         10003040     coredll:COREDLL.dll
 0002:00000044       __imp_LeaveCriticalSection 10003044     coredll:COREDLL.dll
 0002:00000048       __imp_EnterCriticalSection 10003048     coredll:COREDLL.dll
 0002:0000004c       __imp_SetLastError         1000304c     coredll:COREDLL.dll
 0002:00000050       __imp_CeSetPowerOnEvent    10003050     coredll:COREDLL.dll
 0002:00000054       __imp_DisableThreadLibraryCalls 10003054     coredll:COREDLL.dll
 0002:00000058       __imp_GetTickCount         10003058     coredll:COREDLL.dll
 0002:0000005c       __imp_SystemTimeToFileTime 1000305c     coredll:COREDLL.dll
 0002:00000060       __imp_GetLocalTime         10003060     coredll:COREDLL.dll
 0002:00000064       __imp_FileTimeToSystemTime 10003064     coredll:COREDLL.dll
 0002:00000068       __imp_memcpy               10003068     corelib1:COREDLL.dll
 0002:0000006c       __imp_memcmp               1000306c     corelib1:COREDLL.dll
 0002:00000070       __imp_memset               10003070     corelib1:COREDLL.dll
 0002:00000074       __imp___C_specific_handler 10003074     corelib1:COREDLL.dll
 0002:00000078       __imp__XcptFilter          10003078     corelib1:COREDLL.dll
 0002:0000007c       __imp_free                 1000307c     corelib1:COREDLL.dll
 0002:00000080       __imp___security_gen_cookie2 10003080     corelib1:COREDLL.dll
 0002:00000084       __imp_TerminateProcess     10003084     coredll:COREDLL.dll
 0002:00000088       \177COREDLL_NULL_THUNK_DATA 10003088     coredll:COREDLL.dll
 0002:0000008c       __security_cookie          1000308c     corelib0:seccinit.obj
 0002:00000090       __security_cookie_complement 10003090     corelib0:seccinit.obj
 0002:000000a0       ghevReady                  100030a0     battdrvr_mdd:battdrvr.obj
 0002:000000a4       _exitflag                  100030a4     corelib0:cexit.obj
 0002:000000a8       v_imsStart                 100030a8     <common>
 0002:000000ac       v_fStopwatchRunning        100030ac     <common>
 0002:000000b0       v_ftLastChange             100030b0     <common>
 0002:000000b8       v_cmsPreviousCpuUsage      100030b8     <common>
 0002:000000bc       v_fOnExternalPower         100030bc     <common>
 0002:000000c0       v_cmsUsed                  100030c0     <common>
 0002:000000e0       gcsPddBuffer               100030e0     <common>
 0002:00000100       gBatteryContext            10003100     <common>
 0002:00000140       ghevResume                 10003140     <common>
 0002:00000144       gpfnBatteryPddIOControl    10003144     <common>
 0002:00000160       gcsBattery                 10003160     <common>
 0002:00000174       gpPddBufferTemp            10003174     <common>
 0002:00000178       gpPddBuffer                10003178     <common>
 0002:0000017c       gdwPddBufferSize           1000317c     <common>
 0002:00000180       gfExiting                  10003180     <common>
 0002:00000184       ghtBattery                 10003184     <common>
 0002:00000188       __onexitend                10003188     <common>
 0002:0000018c       __onexitbegin              1000318c     <common>
 0002:00000190       _pRawDllMain               10003190     <common>

 entry point at        0001:00001418

 Static symbols

 0001:00001328       _DllMainCRTStartupHelper   10002328 f   corelib0:pegdmain.obj
 0001:00001444       doexit                     10002444 f   corelib0:cexit.obj
